:10000000C9C285C4E2C2E1C2E0C2DFC2DEC2DDC253
:10001000DCC2DBC2DAC2D9C2D8C2D7C2D6C2D5C20C
:10002000D4C2D3C2D2C2040309041803720061000F
:10003000700068006E00650074002E006E006500A0
:1000400074001603470043002F004E0036003400B2
:100050005F0055005300420012011001000000082B
:1000600040177F0500020102000109022200010180
:100070000080320904000001030000000921010191
:10008000000122EC040705810308000A0A0331007D
:10009000300030003000120101010000000840175C
:1000A0007F0500020102030105010905A101850187
:1000B0000901A100050175089506150026FF003508
:1000C0000046FF0009300931093309340935093682
:1000D00081020509150025017501951019012910E6
:1000E000750195108102C0050F0992A102850209D0
:1000F0009F09A009A409A509A615002501350045F9
:100100000175019505810295037501810309941517
:10011000002501350045017501950181020922156F
:1001200001252835014528750795018102C009215F
:10013000A1028501092215012528350145287508E8
:10014000950191020925A1020926092709300931E3
:100150000932093309340940094109420943092890
:10016000250C15013501450C750895019100C00954
:100170005009540951150026FF7F350046FF7F6660
:10018000031055FD75109503910255006600000996
:1001900052150026FF00350046102775089501917D
:1001A0000209531501250835014508750895019187
:1001B000020955A102050109300931150025017513
:1001C0000195029102C0050F09569501910295050E
:1001D00091030957A1020B01000A000B02000A005B
:1001E00066140055FE150026FF00350047A08C0060
:1001F000006600007508950291025500660000C077
:10020000050F09A766031055FD150026FF7F350071
:1002100046FF7F7510950191026600005500C005EC
:100220000F095AA102850209221501252835014529
:1002300028750895019102095B095D150026FF00EC
:10024000350046102795029102095C095E6603108D
:1002500055FD26FF7F46FF7F751091024500660021
:10026000005500C0095FA102850309221501252858
:1002700035014528750895019102092315002501CE
:10028000350045017504950191020958A1020B0141
:10029000000A000B02000A00750295029102C015C7
:1002A00080257F36F0D846102709607508950191A2
:1002B0000236F0D8461027096109629502910215AD
:1002C0000026FF003500461027096309647508956C
:1002D000029102096546102795019102C0096EA19D
:1002E0000285040922150125283501452875089540
:1002F0000191020970150026FF0035004610277590
:100300000895019102096F1580257F36F0D84610B7
:100310002795019102097166140055FE150026FF0C
:1003200000350047A08C00009102097226FF7F462D
:10033000FF7F66031055FD75109501910266000060
:100340005500C00973A1028505092215012528352C
:1003500001452875089501910209701601FF26FFD5
:100360000036F0D8461027751095019102C0097427
:10037000A1028506092215012528350145287508A1
:1003800095019102097509761580257F36F0D846CA
:100390001027750895029102C00968A10285070916
:1003A0002215012528350145287508950191020976
:1003B0006C15002610273500461027751095019101
:1003C0000209691581257F350046FF007508950CE7
:1003D000920201C00966A1028508050109300931B0
:1003E0001581257F350046FF00750895029102C0F2
:1003F000050F0977A102850A092215012528350173
:1004000045287508950191020978A1020979097AB0
:10041000097B15012503750895019100C0097C151C
:100420000026FF00350046FF009102C00990A1029E
:10043000850B0922252815013501452875089501E8
:100440009102C00996A102850C099709980999099A
:100450009A099B099C15012506750895019100C014
:10046000097DA102850D097E150026FF0035004695
:100470001027750895019102C0096BA102850E092C
:100480002215012528350145287508950191020995
:100490006D150026FF00350046FF00750895019197
:1004A00002095166031055FD150026FF7F350046F1
:1004B000FF7F7510950191025500660000C009ABE1
:1004C000A10285090925A102092609270930093158
:1004D000093209330934094009410942094309280D
:1004E000250C15013501450C75089501B100C005B5
:1004F00001093B150026FF01350046FF01750A95ED
:1005000001B1027506B101C0050F0989A10285027A
:100510000922252815013501452875089501B102E4
:10052000098BA102098C098D098E2503150135015E
:10053000450375089501B100C009AC150027FFFF00
:100540000000350047FFFF000075109501B100C0A5
:10055000097FA102850309807510950115003500FA
:1005600027FFFF000047FFFF0000B102098326FFBD
:100570000046FF0075089501B10209A909AA750195
:1005800095021500250135004501B102750695015A
:10059000B103C0C011241FBECFE5D4E0DEBFCDBF84
:1005A00010E0A0E6B0E0E4E2FAE102C005900D92AE
:1005B000A039B107D9F712E0A0E9B0E001C01D925F
:1005C000AE30B107E1F73AD42BCA1ACD85B78260B5
:1005D00085BF8BB780648BBF8BE48093E0008AE596
:1005E0008093DF0008951F93CF93DF936091F00015
:1005F000635067FDCFC08091ED00CCE0D0E0C81B18
:10060000D109CC50DF4F8091EC008D3209F0AEC0A3
:10061000683009F0BDC083EC8093D4008AE58093F4
:100620006000109290008881807621F0CE011CD36A
:10063000AC0184C09A811092DD008981882329F45D
:100640001092DE0042E050E072C0853019F49093C1
:10065000F1006BC0863009F052C08B81813049F4C3
:1006600088E590E09093EF008093EE0042E150E047
:1006700042C0823049F48AE690E09093EF00809384
:10068000EE0042E250E037C0833011F58A818823C2
:1006900049F486E290E09093EF008093EE0044E00E
:1006A00050E029C0813049F48AE290E09093EF0055
:1006B0008093EE0048E150E01EC08230D1F482E425
:1006C00090E09093EF008093EE0046E150E013C07D
:1006D000813249F48CE790E09093EF008093EE0034
:1006E00049E050E008C0823221F4CE014AD2AC0188
:1006F00002C040E050E080E4809390001FC088304A
:1007000029F441E050E023EF30E013C0893019F4C0
:100710009093F3000AC08A3019F441E050E007C01A
:100720008B3019F48BE48093E00040E050E02DED35
:1007300030E03093EF002093EE000DC02FEF4F3FDD
:10074000520749F4888187FF02C04E815F8180E8AB
:100750008093900006C08E819F818417950708F4CE
:10076000AC01509362004093610012C080919000F0
:1007700087FF0EC0CE0114D38F3F21F48EE180930A
:10078000600006C0882321F0109262001092610080
:100790001092F0008091600084FF60C08091610041
:1007A00090916200EFEF8F3F9E0709F457C09C01C4
:1007B0008930910510F028E030E0821B930B909374
:1007C0006200809361008091D40098E8892780932B
:1007D000D400122F222391F16091EE007091EF006E
:1007E0008091900086FF13C09B01C5EDD0E01150B1
:1007F000412F50E01F5FDA01AA52BF4FF9018491E7
:1008000089932F5F3F4FCA17DB07C1F70FC0DB018A
:10081000E5EDF0E01150412F50E01F5F9A012A52A0
:100820003F4F8D918193E217F307D9F7CA010196E3
:10083000860F971F9093EF008093EE0085ED90E078
:10084000612F61D0612F6C5F6C3031F08FEF9FEFC3
:1008500090936200809361006093600094E180B3A4
:10086000857031F49150D9F71092F1001092EB009D
:10087000DF91CF911F9108951F93DC01162F809176
:10088000DF0084FF07C08091E00098E8892780930B
:10089000E00003C08AE58093DF00912FE1EEF0E0F5
:1008A0008D91819391501916DCF381EE90E0612FC8
:1008B0002AD01C5F1093DF001F910895A82FB92F35
:1008C0008FEF9FEF1BC02D918227282F229528277D
:1008D000722F269526952727239526952170782F08
:1008E000892F82272195207C922F22277695279584
:1008F000972782277695279597278227615018F7A3
:10090000809590950895DADF8D939D930895CF9308
:10091000CFB7CF93C395809BE9F7809B09C0809B9D
:1009200007C0809B05C0809B03C0809B01C0A3C003
:10093000DF93C091ED00DD27CC50DF4F809B02C0DC
:10094000DF91EBCF2F930F931F9300B32FEF00FB9B
:1009500020F94F933F9310B34FEF012700FB21F98C
:100960003BE031C04E7F012F10B3216028C0102F13
:100970004D7F2260000000B329C04B7F2460012F0F
:10098000000010B32BC010B3477F28602AC04F7EF1
:1009900000B320612CC04F7D10B320622FC04F7B6D
:1009A00000B3206432C0422700B349934FEF0000E8
:1009B000102710FB20F910B31570C9F1297F91F2AF
:1009C000012700FB21F900B3237F89F2315058F150
:1009D000102710FB22F910B3277E79F2012700FBC4
:1009E00023F92F7C81F200B3102710FB24F92F7913
:1009F00071F200C010B3012700FB25F92F7359F2E3
:100A000000C000B3102710FB26F9223040F200C0CE
:100A100010B3012700FB27F9243028F64F77206810
:100A200010B30000F9CF10E41ABF002719C03B50E3
:100A30003195C31BD04010E41ABF0881033CF9F084
:100A40000B34E9F02091EB001981110F1213EDCF57
:100A50004A81441F093641F10D3211F0013E29F758
:100A60000093F2003F914F911F910F912F91DF91D1
:100A7000CAB7C6FD4FCFCF91CFBFCF911895209168
:100A8000F200222379F31091F000112369F534303C
:100A90006AF13093F0002093EC001091ED003BE000
:100AA000311B3093ED0022C00091F0000130E4F4DE
:100AB0000AE54F7049F43091600034FD19C000938D
:100AC0006000C4EDD0E018C03091DF0034FD10C0EC
:100AD0000093DF00C0EED0E00FC02795A8F451507E
:100AE000A9F4220F0000F9CF4AE503C042ED01C08E
:100AF000432FC4E1D0E032E011B31560909A11BBEE
:100B000002B320E415E05F93012756E002BB27956E
:100B100020F4515021F4220FF9CF012756E00000B4
:100B20003B5A02BBD0F2279528F4515029F4220FEA
:100B30000000F9CF012756E0279502BB20F4515061
:100B400021F4220FF9CF012756E02991332302BB6C
:100B500021F60A7F1091F100110FC651D04002BB5F
:100B600011F01093EB0010E41ABF016011B31A7F6B
:100B7000402F4A7F5F9100C000C002BB11BB42BB47
:100B800071CFFC018081807619F58181863001F575
:100B90008381813019F08232D9F40DC080919500A3
:100BA000909196009093EF008093EE0080919700D3
:100BB000282F30E00FC08091910090919200909387
:100BC000EF008093EE00209193003091940002C0DA
:100BD00020E030E0C9010895E0919800F09199007B
:100BE000309749F00288F389E02D309721F099275A
:100BF00087FD909509950895DC01E0919800F091AA
:100C00009900309751F561307105B9F481E08C930A
:100C10008FE711968C93119712968C9312971396D7
:100C20008C93139714968C93149715968C93159711
:100C300016968C9327E030E015C06230710519F0EC
:100C400020E030E00FC082E08C9311961C92119747
:100C500012961C9223E030E005C00088F189E02D57
:100C600009959C01C9010895DC014DE950E05093BC
:100C7000EF004093EE008C918076803209F071C0D5
:100C800011962C911197223009F440C0233020F4A2
:100C9000213009F066C007C0293009F45FC02A304E
:100CA00009F05FC044C013968C911397813021F0F6
:100CB000833009F053C00AC012966C91662309F480
:100CC0004DC0CA0170E098DF9C014DC012966C9136
:100CD000623061F460939D0020939E0020939F00FA
:100CE0008AE08093A0008093A1000DC06330B1F52D
:100CF00060939D0020939E0020939F008FEF809330
:100D0000A0002093A10025E030E02DC012966C9148
:100D1000862F8150823028F5862F90E08A559F4F8C
:100D20009093EF008093EE0021E030E01CC012961B
:100D3000EC911297EE2339F413968C918093A700CF
:100D40008093A8000EC08E2F8150823050F4F0E0C6
:100D5000EA55FF4F13968C91808303C02FEF3FEF2E
:100D600002C020E030E0C90108958091AA0090916E
:100D7000AB00892B11F410929A0080919A0088237D
:100D800011F42ADF089580919B0087FF02C081E063
:100D900023DF80919C0087FF02C081E01DDF089562
:100DA000FC01662309F448C08081853089F08630D3
:100DB00030F4813049F0843009F03EC010C08930F1
:100DC00019F08A30C9F50FC081818093A90034C021
:100DD0008181813089F5828180939B002CC0828142
:100DE00080939C0028C0643039F5838190E023E033
:100DF000880F991F2A95E1F79093AB008093AA0082
:100E0000818190E08F7790708130910531F0813051
:100E1000910594F00397029778F48281823029F04B
:100E2000833039F0813041F401C081E080939A0031
:100E300002C010929A0099DF81E008952F923F92AC
:100E40004F925F926F927F928F929F92AF92BF92DA
:100E5000CF92DF92EF92FF920F931F93DF93CF9386
:100E600000D0CDB7DEB71A82198214BABB24BA9467
:100E7000B5BAE8EFCE2EC2BA15E011BB78EEE72E78
:100E800070E8F72EC7010197F1F711BA13BF0FE011
:100E900005BD64ECD62ED3BC88EA90E09093920016
:100EA00080939100BAD4909394008093930086E944
:100EB00090E090939600809395006DD18093970079
:100EC00014BAB5BAC2BA11BBC7010197F1F711BA8A
:100ED00013BF05BDD3BCA4D488E190E00FB6F8944D
:100EE000A89581BD0FBE01BD71DB7894BB2477242A
:100EF0007394EE24FF2451E0252E312C40E8642E1B
:100F00003CE2432E31E0532E04C0BB2402C0EE2449
:100F1000FF24A8952FE1E216F10424F01092990025
:100F2000109298008091980090919900892B09F077
:100F300057C080E051DE57DB8CE291E0F20131973F
:100F4000F1F70197D9F71DD58230910539F083303B
:100F5000910589F00197D9F653D401C0A0D2FC01C4
:100F600090939900809398000284F385E02D099571
:100F700080E032DECCCF93D2FC0190939900809335
:100F800098000284F385E02D0995E0919800F09196
:100F900099000488F589E02D09958823E9F480E912
:100FA00091E0F2013197F1F70197D9F71CDB28D4D2
:100FB000FC0190939900809398000284F385E02DC2
:100FC0000995E0919800F09199000488F589E02D49
:100FD0000995882309F49BCF80E0FEDDEE24FF24F1
:100FE000A89501DB772099F0C0DEE0919800F091A0
:100FF00099000484F585E02D0995882321F4772450
:10100000EE24FF2404C00894E11CF11C772408B6E8
:1010100007FE3EC068BEBB2009F03AC0A6DE85B719
:10102000806885BF889585B78F7785BFC201019796
:10103000F1F7E0919800F09199000484F585E02D96
:101040000995882319F4EE24FF2403C00894E11CB9
:10105000F11C00E010E013C068010894C11CD11C11
:101060000684F785E02DC6010995882339F0C10172
:1010700002C0880F991F0A95E2F7B82A8601E0910D
:101080009800F0919900848195810817190724F33D
:1010900008B600FE37C081E088BF8091AA00909119
:1010A000AB00009749F02FEF8F3F920729F001978F
:1010B0009093AB008093AA00E0919800F091990082
:1010C00044815581DE01119620E030E018C0F9011D
:1010D000E955FF4FE081EE2379F08C91853018F0CF
:1010E00085508C9309C0EC93C101022E02C0880F79
:1010F000991F0A94E2F7B82A2F5F3F4F11962417E1
:1011000035072CF3BB2009F404CFCC24DD248B2C31
:10111000992487FC909435C0C4010C2C02C095958D
:1011200087950A94E2F780FF29C08091DF0084FF51
:1011300025C0B6016F5F7F4F8DE990E05DDD00E077
:1011400010E0A82EBB24A7FCB09415C0C80183569C
:101150009F4FB501601B710B6930710514F068E099
:1011600070E08ADB02C03FDAA8958091DF0084FF3F
:10117000FACF085F1F4F0A151B0544F30894C11CE2
:10118000D11CE0919800F091990084819581C81656
:10119000D90614F2BACE82E190E008959093AD00A2
:1011A0008093AC000895009741F0DC01E0EBF0E0A3
:1011B00089E001900D928150E1F7A9EBB0E0E0EBFE
:1011C000F0E089E001900D928150E1F789E090E034
:1011D000089580EB90E069EB70E049E050E00CD4BA
:1011E00008950F931F93DF93CF93CDB7DEB7299761
:1011F0000FB6F894DEBF0FBECDBF1982CE010196A7
:1012000061E070E012D3883109F01FC180E48A8365
:1012100083E08B831C828091AC009091AD00892B80
:1012200011F081E08C838E010E5F1F4FC80163E0D7
:1012300070E0FBD2803409F008C188E0F801119217
:101240008A95E9F74A8120E030E060E870E0F90132
:10125000E65EFE4F8081882339F0CB01022E02C06A
:10126000959587950A94E2F7482B2F5F3F4F2830DA
:10127000310569F74A834B8120E030E060E870E097
:10128000F901EE5DFE4F8081882339F0CB01022EFB
:1012900002C0959587950A94E2F7482B2F5F3F4F40
:1012A0002830310569F740954B834C8120E030E0D0
:1012B00060E870E0F901E65DFE4F8081882339F037
:1012C000CB01022E02C0959587950A94E2F7482B30
:1012D0002F5F3F4F2830310569F74C834D8120E067
:1012E00030E060E870E0F901EE5CFE4F8081882319
:1012F00011F080E007C0CB01022E02C095958795C2
:101300000A94E2F7482B2F5F3F4F2830310559F7F9
:101310004D834E8120E030E060E870E0F901E65C4A
:10132000FE4F8081882339F0CB01022E02C09595B3
:1013300087950A94E2F7482B2F5F3F4F28303105FD
:1013400069F740954E834F8120E030E060E870E01F
:10135000F901EE5BFE4F8081882339F0CB01022E2C
:1013600002C0959587950A94E2F7482B2F5F3F4F6F
:101370002830310569F740954F83488520E030E0FB
:1013800061E070E0F901E35FFE4F8081882339F06E
:10139000CB01022E02C0880F991F0A94E2F7482B56
:1013A0002F5F3F4F2530310569F720E030E060E2E4
:1013B00070E0F901ED5EFE4F8081882339F0CB01AA
:1013C000022E02C0880F991F0A94E2F7482B2F5F64
:1013D0003F4F2330310569F74887498520E030E0E9
:1013E00061E070E0F901EA5EFE4F8081882339F008
:1013F000CB01022E02C0880F991F0A94E2F7482BF6
:101400002F5F3F4F2430310569F7498781E0809392
:10141000B000A1EBB0E0FE01329686E001900D92A3
:101420008150E1F78091AE009091AF00892B29F0B7
:101430008FE78093B5008093B60088858093B700CE
:1014400089858093B80080E001C081E029960FB6BD
:10145000F894DEBF0FBECDBFCF91DF911F910F91EA
:101460000895BFDE90E0882309F491E0892F089564
:10147000B8DE882399F480911301882359F0809174
:101480001401882339F081E090E09093AF008093BD
:10149000AE0008951092AF001092AE00089588EA51
:1014A00090E09093660080936500B7D1E5E6F0E0A8
:1014B00092938293CF01089520918F00253079F087
:1014C000222369F0892B31F0233049F082E08093A8
:1014D0008F000895213019F084E080938F000895E3
:1014E000CF92DF92EF92FF921F93DF93CF930F92F1
:1014F000CDB7DEB785E080938F0010E08CE2C82E78
:1015000081E0D82E7E010894E11CF11C11C0F60187
:101510003197F1F70197D9F71982C70161E070E0BF
:1015200084D1489741F01F5F1F3011F480E004C060
:101530008CE291E0ECCF81E00F90CF91DF911F9191
:10154000FF90EF90DF90CF900895009741F0DC017D
:10155000E2ECF0E089E001900D928150E1F7ABEC14
:10156000B0E0E2ECF0E089E001900D928150E1F70B
:1015700089E090E0089582EC90E06BEC70E049E047
:1015800050E03AD208951F93DF93CF93CDB7DEB7E3
:10159000A6970FB6F894DEBF0FBECDBF1982CE015D
:1015A000019661E070E041D1883119F010928F000E
:1015B00067C080912101882331F080918F008530B0
:1015C00011F410928F0080912101882319F485E095
:1015D00080938F0080918F008230D9F0843081F128
:1015E000882309F044C083E0898380E88A8381E00E
:1015F0008B83CE01049660E870E042E250E009D2AD
:10160000CE01019663E270E010D1882381F184E07D
:101610002CC013E0198380EC8A838BE18B83CE018D
:10162000049661E070E040E250E0F3D1CE01019613
:1016300063E270E0FAD08823D1F010938F0017C0D6
:1016400083E0898380EC8A838BE18B8380E2FE01D7
:101650003496DF011D928A95E9F7CE01019663E287
:1016600070E0E3D0882319F081E080938F0081E05F
:101670008983CE01019661E070E0D7D0803211F00D
:101680008FEFB0C019821A821B821C8240E020E0DA
:1016900030E061E070E0F901E65FFE4F8081882371
:1016A00039F0CB01022E02C0880F991F0A94E2F78D
:1016B000482B2F5F3F4F2430310569F720E030E0A1
:1016C00060E170E0F901EA5EFE4F8081882339F025
:1016D000CB01022E02C0880F991F0A94E2F7482B13
:1016E0002F5F3F4F2430310569F74B838091140100
:1016F00020E0811121E09C81922B809115018111C4
:1017000082E0892B8C83498120E030E060E870E042
:10171000F901E65EFE4F8081882339F0CB01022E6D
:1017200002C0959587950A94E2F7482B2F5F3F4FAB
:101730002830310569F749834A8120E030E060E8CC
:1017400070E0F901EE5DFE4F8081882339F0CB0116
:10175000022E02C0959587950A94E2F7482B2F5FD9
:101760003F4F2830310569F74A8381E08093C200FA
:10177000898181588093C3008FE7982F941B9093A1
:10178000C4008093C5008093C6008093C7008093F7
:10179000C8008B818093C9009C819093CA0080917E
:1017A0000E01882319F094609093CA0080910F0174
:1017B000882329F08091CA0088608093CA008091B4
:1017C0001001882329F08091CA0080618093CA00AB
:1017D00080911101882331F08091CA00806280934A
:1017E000CA0080E0A6960FB6F894DEBF0FBECDBF4C
:1017F000CF91DF911F910895A09AA898C4DE089513
:1018000088EA90E090937C0080937B0006D0EBE721
:10181000F0E092938293CF0108958CEE94E00895C6
:10182000A598AD98BC9AC4980895EF92FF920F9333
:101830001F93CF93DF937C01662309F44FC070E0C0
:1018400020E030E0E0E0F0E011C088818423FD0179
:10185000E65FFE4F808311964695A017B107A9F762
:101860002F5F3F4F2617370754F4FD01DF0140E893
:10187000E701C20FD31F8F01085F1F4FE6CFEAE0D9
:10188000F1E0CF93DF93EF93FF930191002311F0E9
:1018900049F416C00000A59A19E00FD0A598119739
:1018A000A1F70EC0A59A11E008D0A59815E005D0C3
:1018B00000000000119749F703C01A95F1F7089549
:1018C0000000FF91EF91DF91CF91A59A11E0F5DF34
:1018D000A5980FEF0A9511F09D9BFCCFEAE0F1E08F
:1018E000EF93FF93112700270395A1F09D99FCCF5B
:1018F00008C004E6039572F09D99FCCF139551F052
:10190000019304E6039532F09D9BFCCF139511F0F3
:101910000193EFCFFF91EF91612F70E06115710599
:1019200031F110FF24C040E050E020E030E00CC076
:101930008081F901E75FFE4F9081E0E0891708F4AC
:10194000E1E0EC934F5F5F4FDA01A65FBE4FF90114
:10195000E65FFE4F2E5F3F4F411750F384E18A95BB
:10196000F1F79B01215030403595279502C020E0CA
:1019700030E0C901DF91CF911F910F91FF90EF905F
:101980000895DF93CF930F92CDB7DEB71982CE01C2
:10199000019661E070E049DF009719F420E030E043
:1019A00026C0489711F580910E01882311F098E028
:1019B00001C090E080910F0181119460809110012D
:1019C0008111926080911101811191609A3028F407
:1019D000983028F4953049F405C09B3031F422E06A
:1019E00030E005C021E030E002C023E030E0C90172
:1019F0000F90CF91DF910895FB01DC0104C08D9120
:101A00000190801921F441505040C8F7881B990B70
:101A10000895DC0101C06D9341505040E0F70895F6
:041A2000F894FFCF68
:101A24005AFFFF00000000010000000000380AF126
:101A340008E908D308CE08310A00000000010000BC
:101A4400000000FC0BC30ABB0AA50A5C0A700A0565
:00000001FF
